:100000008CC0B2C081C3B0C0AFC0B3C0ADC0ACC0C3
:10001000ABC0AAC0A9C0A8C05CC1A6C0A5C081458C
:1000200086468B479048944997609B619E62A16386
:10003000A464A765AA66AC67AE68B069B280B481F3
:10004000B682B883BA84BB84BD84FF21000000005F
:100050000000000000000000000023456C98C9FF6C
:10006000040714233764A0FFFFFFFFFFFFFFFFFF1C
:10007000FFFFFF00000000000000000023405F7A47
:10008000B4FFFFFFFFFFFF001400081400080E1468
:100090000004080E14000305080E140004080A0EDC
:1000A0001114000305080A0E1014000305080A0EB7
:1000B0001012140008000E00080E0004080E0003C1
:1000C00005080E0004080E1100080E1100F3F404D8
:1000D000080E10121400080A0C0E0F10121400085B
:1000E0000EED14000203040500041400040E1400B5
:1000F000040810140004080F1114000305080A0E68
:100100000004080A0E00EEEDECEB140E08040004E7
:10011000080E00EBECEDEEF3F41411241FBECFE556
:10012000D1E0DEBFCDBF20E0A0E6B0E001C01D926F
:10013000AA37B207E1F7EBE7F0E085E5808781E0D9
:10014000838314821282868311828BE0818788E503
:100150008287E1E6F0E08DEF87838EEF8583712C57
:1001600055245A94B7D0EBC24BCF1BBC19BC18BC5A
:100170000895189525B7277E25BF29B7226029BF86
:1001800021E022BF019728F020E188952150E9F76E
:10019000F9CF089588EE93E0EDCF369A3699FECFE9
:1001A00095B18091600089270895CF93C72D81E094
:1001B000870D8F73782E662D90E0B3D26FEF8C2F62
:1001C00090E0CF91AEC2FF920F931F93CF93DF9336
:1001D000F82E0CE710E0CEE7D0E0F11005C0CE011C
:1001E00098D2F801808304C0F8016081CE0199D2D1
:1001F00021970F5F1F4FC437D10579F7DF91CF915A
:100200001F910F91FF900895D0DF81E0DCCF811125
:1002100001C0ABCF815090E0FC01E45BFF4FE49163
:10022000EBBDFC01E05AFF4FE491E9BDFC01EC5845
:10023000FF4F849188BD08950F931F93CF93C82FCC
:100240008B01CC2359F085E0E2DFC80193DF8DDF1D
:10025000C80190DFC8018EDFC150F3CFCF911F914D
:100260000F910895EF92FF920F931F93CF93C8E0E1
:10027000E82EF12C062F10E084E1C9DFC7017ADFF8
:1002800074DFC80177DFC150B9F7CF911F910F918B
:10029000FF90EF9008951F93CF93DF938FEA87B974
:1002A00086EC86B91092600010E1C0E0D0E085E0F5
:1002B00090E060DF72DFC80FD11D1150C1F7CE0191
:1002C00024E0969587952A95E1F7DF91CF911F91CC
:1002D0000895189510927A0087E790E01AD2853534
:1002E00019F0612C91DF11C0712C872D90E011D293
:1002F000682E8F3F19F080E066DF07C0872D91E000
:10030000970D792E803488F3F6CF20918400C09128
:100310007E0010917F0080917C00882319F010E00E
:10032000C0E02AE12F5F90E040E050E0A8E8B0E0B4
:10033000222379F0BD016F5F7F4FFB013197E4917C
:10034000EE2319F0962F9A1BF6CF2150AD01DB0159
:10035000EFCF092F6C2F70E0A92FB0E0E02FF0E075
:10036000112321F09D012E1B3F0B05C09F01215041
:100370003109260F371F3197E40FF51FF4902659E6
:100380003F4FF901F082015049F79C0F909386008E
:10039000CC2371F0112329F0292F30E021503109AD
:1003A00002C020E030E0F901E659FF4F41E0408310
:1003B00027E0290F322F3150E32FE91BF0E0ED5EEB
:1003C000FE4FE491A32FB0E0A659BF4FEC93391331
:1003D000F2CFE22FF0E0E759FF4F31E050916A0091
:1003E0004081541330E0231B20938700362D353F86
:1003F000E8F5452D4330B0F4809188008F3F29F413
:1004000080917A008093880006C081E0860D682E76
:10041000891708F0612C809188008F5F8F7180931D
:10042000880024C030917A00309388004730C0F4AF
:1004300030918100332311F0882339F081E0860D5B
:10044000682E891798F0612C11C0862D6916D9F392
:10045000662019F08150682E09C02150622E06C016
:100460008111F1CF80917D00882369F3512C8FEFAA
:100470008DBD80E68CBDAA9A8FE384BB83E187BBE8
:1004800088EE88BB81E083BF91EA9ABD80BF8BB7BD
:1004900080628BBF8AB785608ABF85B7806285BF5F
:1004A00078948CE287B986EC86B93699FECF8FEFC7
:1004B00080936000C62DC53F10F0612C3CC0809138
:1004C0008800803138F4E62DF0E0E659FF4FC08116
:1004D000DC2F31C05FDE80917A0080938800CCE70A
:1004E000D0E000E010E0FF24F39481E0800F0F5F84
:1004F0001F4F98819F3F29F4219608301105A9F7D5
:10050000E2CF6DE570E098DEF801EF59FF4F6080B3
:1005100088818F25888378DE6FE070E080E28CDE52
:1005200088818F258883612C6FDE34DE80917C008A
:10053000882311F3C8CF39DE10E0F12C8CE2D82EDD
:1005400096ECC92EEE24EA94CE3E19F463E481E2DF
:1005500004C0CD3E21F468E284E184DE76C0CC3E66
:1005600011F469E203C0CB3E19F462E581E0F5CFF6
:10057000C33F81F404E084E14ADE85E090E0FADDE7
:1005800088E045DE81E490E0F5DD0150A1F780EDE3
:1005900092E05AC0C43F51F584E690E0EBDDFDDD0A
:1005A00090E0292F30E0F901E25EFF4FE491E81777
:1005B00010F49E5FF6CFF901E15EFF4F04916DE705
:1005C00070E0802F82958695877036DE8EEE92E001
:1005D000D1DD65E070E081E02FDE85E694E0CADDE4
:1005E0006DE770E0802F8F7127DE0DC0CE3F71F474
:1005F00000E00093840008DE6AEF70E081E01CDE1A
:100600000F5F0A31B1F7C6DDC5DD1FC0CD3F69F50B
:100610008FEF80938500F8DD85E0F9DDBBDDBADD85
:1006200084E1F5DD38DE80938500EEDDB3DDB2DDFB
:10063000F9CF3699FECFE0926000F3949091850057
:100640008917C8F484EF91E095DD80917A0080935A
:100650008800A3DD803998F51F5F183008F474CF47
:10066000D53190F010E0DAE0CAE08D2FD0DD13DE56
:10067000D7B8C6B8DECFDB3028F3F4E1FF1510F7AA
:10068000E0927A00DAE0DECFD23030F08D2F86951E
:100690008695D695D80F12C068DD85B7877E8061B4
:1006A00085BFF89485B7846885BF8B7F85BF85B784
:1006B000806285BF889585B78F7D85BFCD2F10E07F
:1006C00043CF112416B851DD87B38C7E87BB94E4E9
:1006D000B29914C05394999885B7877E806185BF7D
:1006E000A89591BD85B7846885BF8B7F85BF7894B9
:1006F0008895F89481B58F7B81BDEACF8FE58DBF5A
:1007000081E08EBF1FBEE6DD552011F0189501C0B7
:10071000D8DFE199FECF1FBA8EBBE09A99278DB33F
:100720000895262FE199FECF1CBA1FBA8EBB2DBBB0
:100730000FB6F894E29AE19A0FBE01960895F894E4
:02074000FFCFE9
:00000001FF
